:100000000C94FB060C9442070C9442070C94392A7A
:100010000C9442070C9442070C9442070C9442073C
:100020000C9442070C9442070C942A270C94DF2569
:100030000C94A51C0C9442070C9442070C944207A4
:100040000C9442070C9442070C9442070C9442070C
:100050000C9442070C94331C0C9442070C944207F6
:100060000C9442070C9442070C9442070C944207EC
:100070000C9442070C9442070C9442070C944207DC
:100080000C9442070C9442070C9442070C944207CC
:100090000C9442070C9442070C9442070C944207BC
:1000A0000C9442070C9442070C9442078610861069
:1000B000C810C810EC100A11C712C7124C11C71291
:1000C0003B123B12A714A914B414AB14AD14AF1413
:1000D000B114B314B614B814BA14C514BC14BE14B5
:1000E000C014C214C414C714E7200E21B0220E217C
:1000F000B02256217921B02274228722B923B92354
:10010000CB23CB23C223CB23CB23CB23B923B923AC
:10011000C723CB23CB23C72300000000000000002F
:1001200000000101010101010101010202020202BC
:10013000020202030303030303030404040404058B
:100140000505050506060606060707070708080849
:10015000080909090A0A0A0B0B0B0C0C0C0D0D0DF2
:100160000E0E0E0F0F101010111112121313141483
:10017000151516161717181819191A1A1B1C1C1DF5
:100180001D1E1F1F20212122232324252526272849
:1001900028292A2B2C2C2D2E2F3031313233343577
:1001A000363738393A3B3C3D3E3F40414243444577
:1001B000464748494B4C4D4E4F5052535455575853
:1001C000595A5C5D5E606163646567686A6B6C6EFA
:1001D0006F7172747677797A7C7D7F81828486876D
:1001E000898B8D8E9092949597999B9D9FA1A2A4A7
:1001F000A6A8AAACAEB0B2B4B6B9BBBDBFC1C3C5A8
:10020000C8CACCCED0D3D5D7DADCDEE1E3E6E8EA63
:10021000EDEFF2F4F7F9FCFF2223252628292A2CFA
:100220002D2F3032333536383A3B3D3E4042434540
:1002300047494A4C4E5051535557595A5C5E60627B
:10024000646668696B6D6F71737577797B7D7F818B
:10025000838587898A8C8E90929496989A9C9E9F8B
:10026000A1A3A5A7A8AAACAEAFB1B3B4B6B8B9BBA9
:10027000BCBEBFC1C2C3C5C6C7C9CACBCCCDCED018
:10028000D1D2D2D3D4D5D6D7D7D8D9D9DADADBDB05
:10029000DBDCDCDCDCDCDDDDDDDDDCDCDCDCDCDB9C
:1002A000DBDBDADAD9D9D8D7D7D6D5D4D3D2D2D1E5
:1002B000D0CECDCCCBCAC9C7C6C5C3C2C1BFBEBCD8
:1002C000BBB9B8B6B4B3B1AFAEACAAA8A7A5A3A149
:1002D0009F9E9C9A98969492908E8C8A898785830B
:1002E000817F7D7B79777573716F6D6B69686664EB
:1002F00062605E5C5A5957555351504E4C4A4947BB
:10030000454342403E3D3B3A3836353332302F2D5F
:100310002C2A29282625232200AF290014001A00A0
:1003200009001300050000002B430400150016000F
:1003300017000A000000F05C1D001B00060007000B
:1003400019000000000000000000F25CD75C2C44A3
:1003500000002A0033001C0018000F000D000000F0
:10036000340012000C000800110010000000F15CC5
:100370003800370036000B000E00000000000000BF
:100380000000F35CD85C055800000100010001008A
:1003900001000100010000002B000100010001002C
:1003A000010001000000E000010001000100010067
:1003B00001000000000000000000E200E1002C420B
:1003C0000000010001000100010001000100000027
:1003D0000100010001000100010001000000010016
:1003E0000100010001000100010000000000000008
:1003F0000000E700E5000100000035001E001F00BE
:1004000001002000210000002F0030000100010049
:1004100001003100000022002300240025002600F6
:1004200027000000000000000000010001000100A2
:1004300000004C003E003D003C003B003A00000044
:10044000010043004200410040003F00000028003E
:1004500001002E002D0045004400000000000000B7
:100460000000010001000100000029003A003B00EB
:100470003C003D003E00000001003F004000410004
:1004800042004300000001004400450048004900CC
:1004900046000000000000000000010001002C00E8
:1004A000000055005400610060005F005300000030
:1004B000570056005E005D005C00390000005800E7
:1004C00067005B005A005900470000000000000070
:1004D00000002A0063006200000035001E001F00BB
:1004E000200021002200000035021E021F0220020F
:1004F000210222020000010000000000000022147E
:1005000000000000000000000000010001000100E8
:1005100000003100270026002500240023000000F1
:1005200031022E022D0025022402230200000100C8
:100530002E00370236022D020000000000000000ED
:100540000000E7000100010000003500F9002B0366
:10055000F0002B01F50000002B00FA00F200F10082
:10056000F300F400000001000000FB000000FC00AC
:100570000000000000000000000001000100010078
:1005800000004C0000004D0052004A004B000000EB
:10059000000000004F00510050004E00000001001C
:1005A0000000FF00FE00FD00000000000000000051
:1005B0000000E700010005510000005C0000AD00F4
:1005C000A900AB0000000000F75C0000AC00AA002E
:1005D000AE00000000000000A6000000A80000001F
:1005E0000000000000000000000001000100010008
:1005F0000000C55CC65C0000000001520052000013
:10060000C75CC85CD05CCF5CCE5CCD5C0000C95CD4
:10061000CA5C000000000000C25C00000000000096
:100620000000010001000100000000DA02818FD902
:10063000F1DB40A4A62EAF00A0C000A1C800AED53B
:1006400080A81FD300408D142000202020202000EF
:10065000205343524C0020202020200020434150B2
:100660005300202020202000204E554D2000202027
:1006700020202000444F434B20004D6F64653A0A10
:10068000000A002020202020004155582020002072
:1006900020202020004655454C20002020202020EE
:1006A0000050524F4720000A00556E6B6E200055D7
:1006B00074696C20004578742020004779726F209F
:1006C00000436F6D6D20005374616765002020202A
:1006D0002020000A0047414D452000434C4D4B204F
:1006E00000808182838485868788898A8B8C8D8E21
:1006F0008F9091929394A0A1A2A3A4A5A6A7A8A924
:10070000AAABACADAEAFB0B1B2B3B4C0C1C2C3C49A
:10071000C5C6C7C8C9CACBCCCDCECFD0D1D2D3D411
:100720000000AE643214783C1E1E140A050501094F
:1007300002A10185020901A1000509190129051578
:10074000002501950575018102950175038101055B
:1007500001093009311581257F9502750881060947
:10076000381581257F950175088106050C0A380228
:100770001581257F950175088106C0C00501098096
:10078000A10185031601002603001A81002A8300B7
:10079000751095018100C0050C0901A101850416A1
:1007A0000100269C021A01002A9C02751095018105
:1007B00000C005010906A1018505050719E029E723
:1007C0001500250195087501810205081901290503
:1007D00095057501910295017503910105071900B1
:1007E00029EF1500250195F075018102C005010969
:1007F00006A101050719E029E715002501950875EF
:1008000001810295017508810105081901290595E5
:1008100005750191029501750391010507190029DC
:10082000FF150026FF00950675088100C009023BF0
:1008300000020100A0FA09040000010301010009FF
:1008400021110100012240000705810308000A0967
:10085000040100010300000009211101000122C070
:10086000000705820320000A1201100100000008A1
:10087000EDFE6030010001020301040330000000BE
:100880001E0343006F0072006E00650020004B00E5
:100890006500790062006F00610072006400000072
:1008A000100366006F006F007300740061006E003B
:1008B0000000040309040000000000003E5B4F5BE1
:1008C0003E003E6B4F6B3E001C3E7C3E1C00183CC5
:1008D0007E3C18001C577D571C001C5E7F5E1C0070
:1008E00000183C180000FFE7C3E7FF0000182418B9
:1008F0000000FFE7DBE7FF0030483A060E0026293C
:1009000079292600407F05050700407F05253F0027
:100910005A3CE73C5A007F3E1C1C0800081C1C3E49
:100920007F0014227F2214005F5F005F5F000609D2
:100930007F017F00006689956A00606060606000EA
:1009400094A2FFA2940008047E04080010207E20D8
:10095000100008082A1C0800081C2A0808001E109D
:10096000101010000C1E0C1E0C0030383E383000E9
:10097000060E3E0E060000000000000000005F00B2
:100980000000000700070000147F147F1400242AD1
:100990007F2A120023130864620036495620500053
:1009A000000807030000001C224100000041221C37
:1009B00000002A1C7F1C2A0008083E08080000804E
:1009C000703000000808080808000000606000009F
:1009D0002010080402003E5149453E0000427F407D
:1009E00000007249494946002141494D330018141D
:1009F000127F10002745454539003C4A49493100DE
:100A0000412111090700364949493600464949291B
:100A10001E00000014000000004034000000000828
:100A2000142241001414141414000041221408006C
:100A30000201590906003E415D594E007C12111217
:100A40007C007F49494936003E41414122007F41B7
:100A500041413E007F49494941007F0909090100A0
:100A60003E41415173007F0808087F0000417F41EB
:100A700000002040413F01007F08142241007F40D8
:100A8000404040007F021C027F007F0408107F006E
:100A90003E4141413E007F09090906003E41512186
:100AA0005E007F09192946002649494932000301A1
:100AB0007F0103003F4040403F001F2040201F00B7
:100AC0003F4038403F006314081463000304780477
:100AD00003006159494D4300007F41414100020438
:100AE00008102000004141417F000402010204007F
:100AF0004040404040000003070800002054547864
:100B000040007F2844443800384444442800384496
:100B100044287F0038545454180000087E0902000D
:100B20001824241C78007F080404780000447D40C9
:100B300000002040403D00007F102844000000419C
:100B40007F4000007C04780478007C08040478006E
:100B50003844444438007C182424180018242418ED
:100B60007C007C0804040800485454542400040405
:100B70003F4424003C4040207C001C2040201C00BE
:100B80003C4030403C004428102844004C90909059
:100B90007C004464544C44000008364100000000CE
:100BA0007700000000413608000002010204020044
:100BB0003C2623263C00000000000000000000004E
:100BC00000E0381C0C0603030101010101010303CD
:100BD0008286CCF8F0F0381C0C0000000000000009
:100BE00000000000000000000000C070F80C04C607
:100BF000A2B39F8701011F6666444C5870E08000D5
:100C0000000000000000000000000000000000C024
:100C1000E078188CC6E6E3E3C38303037376760CAF
:100C200018F8F0C000000000000000000000000004
:100C300000000000E0F0F0F0E0ECEEF7F3702000D0
:100C40007C7C7C7E007E7E7E7F7F7F000080C0E09B
:100C50007E5B4F5BFEC00000C000DCD7DEDEDED76F
:100C6000DC00C000000000000000000000000000E8
:100C70000000000000000000000000000080C040F4
:100C80007FF36020303038189CCC6C6E3E3E1F0FD6
:100C90000F030301C0FF3E00000000000000000041
:100CA0000000000000000000007FC1001D67C08040
:100CB000010000F00F0000000C1A32C201C1FF3E1B
:100CC00000000000000000000000000000007EFFA7
:100CD000800000C3C7C78F0F070380C0C0C0C0809B
:100CE00000070FFF7F000000000000000000000070
:100CF000000000000F1F3F7F7F7F7F7F3F1E0C00A3
:100D00001F1F1F3F003F3F3F7F7F7F00307B7F786B
:100D100030202030787F3B0003000F7F0F0F0F7FC4
:100D20000F000300000000000000000000000000B1
:100D30000000000000000000000000000101004071
:100D400060313B1E0C1E3623616060606060603065
:100D50001C3E3E3F1D00000000000000000000009F
:100D60000000000000000000000001070C18103314
:100D70003E386E67606060203018080F0603000080
:100D80000000000000000000000000000000000162
:100D900003060C1931216060606061636767333955
:100DA000180E070300000000000000000000000013
:100DB0000000000000000000000000000000000033
:100DC0000000000000000000000000000000000023
:100DD0000000000000000000000000000000000013
:100DE0000000000000000000000000000000000003
:100DF00000000000000011241FBECFEFDAE0DEBFCC
:100E0000CDBF04B603FE27C08091E9049091EA04A7
:100E1000A091EB04B091EC048730904BA740B04B0D
:100E2000D1F41092E9041092EA041092EB041092AB
:100E3000EC0414BE84B7877F84BF0FB6F894A895DE
:100E400080916000886180936000109260000FBE06
:100E5000E0E0F8E3099524E0A6E5B1E001C01D92C9
:100E6000A93EB207E1F711E0A0E0B1E0E0EBF9E55F
:100E700002C005900D92A635B107D9F70E94AA15B8
:100E80000C94D62C0C9400000895AF92BF92CF9290
:100E9000DF92EF92FF920F931F93CF93DF93F82E81
:100EA000E62EE901E42FF0E0611106C0E85EFE4F96
:100EB0008491E82F482F7BC0062F10E026E0829F08
:100EC000C00111242FEF30E0B9010E948E2C5BEAA3
:100ED0005603C001579F900D11248F0D911D8F0D4A
:100EE000911D982F990F890F6901C01AD10ACE9EC2
:100EF000D001CF9EB00DDE9EB00D11249B2FE89E39
:100F000070011124EF2CFF246901CE18DF08CE9E5A
:100F10007001CF9EF00CDE9EF00C11245901A81A2E
:100F2000B108A09E6001A19ED00CB09ED00C1124EF
:100F30000D2D1127201B310B2E9F80012F9F100D8F
:100F40003E9F100D1124812F6230710591F048F4FD
:100F500061157105E9F061307105C1F4842F4F2DE1
:100F600017C06430710571F040F06630710581F092
:100F70000DC0842F4B2F912F0BC0E42F4B2F9E2F92
:100F80008F2D06C08B2F942F412F02C08B2F9F2DAA
:100F9000E42FF0E0E85EFE4F4491E82FF0E0E85ED9
:100FA000FE4F8491E92FF0E0E85EFE4FE491498323
:100FB0008883EA83DF91CF911F910F91FF90EF908B
:100FC000DF90CF90BF90AF9008959091CA0192FFAB
:100FD0000DC0282F2871283019F4877F846006C03F
:100FE000282F2471243011F48B7F886093FF0DC06B
:100FF000282F2871283119F4877E846106C0282F94
:101000002471243111F48B7E886194FD877E0895CC
:101010001F93CF93DF93CDB7DEB767970FB6F894E2
:10102000DEBF0FBECDBF4B8B5C8B6D8B7E8B8F8BF2
:101030006E897F896115710531F05F3F31F481E080
:101040004F3F19F403C081E001C080E080FD09C07A
:101050008091B2019091B30101969093B301809376
:10106000B20186E09E01235F3F4FD901E82F1D9218
:10107000EA95E9F795E0FE017396D90101900D928A
:101080009A95E1F74D875E87798B688BF901DE01D0
:10109000179601900D928A95E1F7CE0107960E946E
:1010A000D42381113EC086E0FE013796DE01119601
:1010B00001900D928A95E1F7FF81E8856A857B852D
:1010C0006115710531F0EF3F31F481E0FF3F19F414
:1010D00003C081E001C080E080FD23C02091AB040B
:1010E00030E0C9010196877099274091DC0450E0F7
:1010F0008417950779F1F983EA837D836C8396E001
:10110000929FD001939FB00D1124A455BB4FFE01B7
:10111000319601900D929A95E1F78093AB040E946D
:10112000392316E08091DC049091AB04891709F112
:10113000189FC001112484559B4F0E94D4238823FB
:10114000C1F08091DC0490E001968770992780932C
:10115000DC04E8CF10926B020E94A4251092AB042D
:101160001092DC04E5EAF4E086E0DF011D928A9546
:10117000E9F767960FB6F894DEBF0FBECDBFDF91DB
:10118000CF911F9108952091AE013091AF012817A2
:10119000390771F09093AF018093AE01E091CC01DB
:1011A000F091CD01309721F00084F185E02D099474
:1011B00008952091AC013091AD012817390771F0E5
:1011C0009093AD018093AC01E091CC01F091CD0101
:1011D000309721F00680F781E02D09940895E09181
:1011E000CC01F091CD01309721F00190F081E02DFC
:1011F000099480E008958091DF0480FF0AC0539A2B
:101200008BB1877F9BB198602FB7F894E9E5F1E047
:101210000BC0E9E5F1E0118210821282339631E0D1
:10122000EA3AF307C1F7EBCF31E0EA3AF30789F086
:10123000319148E09BB9000000C037FF8BB9330FF4
:10124000000000C000C000C08BB900C04A9591F7F3
:10125000EBCF2FBF87EC90E00197F1F700C00000C3
:101260000895EF92FF921F93CF93DF93EC0189E5EE
:10127000E82E81E0F82E10E04091E204493708F0B2
:1012800048E78C8197016091E104810F0E94450736
:10129000175F83E0E80EF11C133F71F70E94FB0813
:1012A0009A818C8190FF02C08F5F01C081508C8336
:1012B000DF91CF911F91FF90EF9008959091DF04FF
:1012C00090FF0CC0E9E5F1E08183608342833396AF
:1012D00091E0EA3AF907C1F70C94FB080895CF931F
:1012E000DF9300D01F92CDB7DEB79091DF0490FF5F
:1012F0000DC0493708F048E79E012F5F3F4F0E941D
:1013000045074B8169818A810E945E090F900F9089
:101310000F90DF91CF910895CF93DF93EC01EFED24
:10132000F4E0438162818C810E946F098C818F5F20
:101330008C83DF91CF910895CF93DF93EC01EC8103
:10134000F0E0E85EFD4F4491EFEDF4E062818181D1
:101350000E946F098C818F5F8C83DF91CF910895FC
:101360008091DF0480FF02C08695089580E0089593
:101370008091DF04282F269530E02115310519F4DE
:101380008170826005C02F30310524F081708C613E
:101390008093DF048091E204893718F088E7809316
:1013A000E2040895CF92DF92EF92FF926B017C01ED
:1013B0000E94B809B701A60188E090E0FF90EF9085
:1013C000DF90CF900C94602CEF92FF920F931F93BD
:1013D000CF93DF9300D01F92CDB7DEB7082FF62E44
:1013E000142FE22E8091DF0480FF39C0E82FE695AC
:1013F000F0E0E95CFE4F908190931F028E7F823077
:1014000081F4493708F048E79E012F5F3F4F6F2D69
:10141000802F0E9445074B8169818A810E945E0965
:101420000CC0923019F41091E20407C0963019F400
:101430000091E00402C09930D9F30093E004F092E7
:10144000E1041093E204EE2051F06091DF0470910A
:10145000E0048091E1049091E2040E94D2090F908F
:101460000F900F90DF91CF911F910F91FF90EF9010
:101470000895EFEDF4E083E0808311828FEF8283A3
:1014800088E78383148260817181828193810C94C7
:10149000D209CF93DF9328E3829FC0011124FC017E
:1014A00037E0739FE00DF11D1124E60FF11DEE0FE3
:1014B000FF1FE65EFC4FC591D491CE01C238D10525
:1014C00049F1B0F4C133D10509F464C048F4C9321C
:1014D000D10509F458C0CA32D10509F462C068C008
:1014E000C533D10509F448C0C933D10599F060C0AE
:1014F000C33ED10541F138F4C03ED10591F0C23E62
:10150000D105B1F055C0C63ED10521F1C73ED10588
:1015100061F14EC02091CA0120FD09C221FD07C220
:1015200008C22091CA0120FF04C289E390E001C2F1
:101530002091CA0122FFFDC18091CA0184FDA9C189
:1015400083EE90E0F6C18091CA0182FFF5CF82EE72
:1015500090E0EFC12091CA0123FFEBC18091CA0145
:1015600084FD97C187EE90E0E4C18091CA0183FFBA
:10157000F5CF86EE90E0DDC12091CA0125FFD9C1EB
:1015800089E290E0D6C12091CA0125FFD2C185E34E
:1015900090E0CFC12091CA0126FFCBC18AE290E042
:1015A000C8C12091CA0126FFC4C181E390E0C1C136
:1015B000C11540E5D40708F049C0C11520E4D207A1
:1015C00008F030C1C83ED10520F5C03ED10508F075
:1015D000B0C1C83AD10570F4C53AD10508F0ADC024
:1015E000C130D10509F4A5C108F453C1249708F40A
:1015F00050C19FC1CF3BD10508F4AAC0C03CD10562
:1016000008F447C1CE01880F991FFC01E856F0404D
:10161000FEC0C11530E2D30760F4C11541E0D40724
:1016200008F087C1C03FD10508F433C1CE019065F1
:1016300080C1C11580E3D80708F0ECC0CE019F70CF
:10164000FC01EE0FFF1FE85EFE4FE1C0C11525E56E
:10165000D20708F045C0C11534E5D30708F0FAC039
:10166000C11542E5D40718F5C11581E5D80708F082
:10167000DDC0CE0174E0969587957A95E1F7282F25
:1016800023703C2F337081E090E002C0880F991FD7
:101690003A95E2F79C68922BEC2FEF70E695E69571
:1016A00020E2E29FF00111248E2B9F2B42C1AE015C
:1016B000437055272C2F26952695C115D34508F044
:1016C000BAC081E090E002C0880F991F4A95E2F706
:1016D00040E2249F90011124822B932B9C6829C106
:1016E000C11549E5D40798F4C11588E5D80708F075
:1016F000B6C0C11526E5D20708F0CBC08C2F0E94DA
:10170000E5078F7190E0982F8827906212C1C1156C
:101710003AE5D30708F4A8C0CE019056811590424F
:1017200008F0B7C08D2F8F710E94E507FE01FF27DB
:10173000F0628F719F01382BAAC0C53AD10509F418
:10174000ABC0C63AD10509F0AAC082E890E4F1C066
:10175000C83AD10509F4A6C0C93AD10509F4A5C013
:10176000CA3AD10509F4A4C0CB3AD10509F4A3C003
:10177000CC3AD10509F4A2C0CB3BD10509F4A1C0F4
:10178000CC3BD10509F4A0C0CD3AD10509F49FC0E6
:10179000C03BD10509F49EC0CE3AD10509F49DC0E5
:1017A000CF3AD10509F49CC0C13BD10509F49BC0D7
:1017B000C23BD10509F49AC0C33BD10509F499C0D5
:1017C000C43BD10509F498C0C53BD10509F497C0C5
:1017D000C63BD10509F496C0C73BD10509F495C0B5
:1017E000C83BD10509F494C0C93BD10509F493C0A5
:1017F000CD3BD10509F492C0CE3BD10509F491C08F
:10180000CA3BD10509F490C080E094E492C0859170
:1018100094918FC0CE019927D3FF02C0986C89C0E4
:10182000906C87C0CE019F70906A83C09C2F8827E0
:10183000816F906A7EC081E090E002C0880F991F9E
:101840004A95E2F740E2249F90011124822B932BCA
:101850009A686FC09C2F8827846F906A6AC09C2FFB
:101860008827806F906A65C08C2F8F700E94E50773
:10187000FE0194E0F695E7959A95E1F7EF70F0E0B8
:10188000FE2FEE27F06A8F70806E9F01282BC90112
:1018900050C080E090E04DC081E890E44AC083E809
:1018A00090E447C082EE94E444C089EE94E441C0E1
:1018B0008AEE94E43EC085EB94E43BC086EB94E46E
:1018C00038C083EB94E435C084EB94E432C087EBFA
:1018D00094E42FC08CEC94E42CC08DEC94E429C0EB
:1018E00083E895E426C08AE895E423C082E995E47C
:1018F00020C084E995E41DC081E296E41AC083E229
:1019000096E417C084E296E414C085E296E411C020
:1019100086E296E40EC087E296E40BC08FE694E47C
:1019200008C080E794E405C08AE296E402C080EE35
:1019300090E0DF91CF910895CF93DF93AFE2B1E0D4
:1019400043E351E061E070E08D91E82FE295EF70A4
:10195000F0E021A18F70EB0102C0CC0FDD1F8A9552
:10196000E2F7CE019C2F9095922391A392A1892B0F
:1019700082A34A175B0741F7DF91CF9108959F92A9
:10198000AF92BF92CF92DF92EF92FF920F931F938D
:10199000CF93DF9380910401811103C0C4E0D0E0B4
:1019A00002C0C0E0D0E0AE014F535E4F7A018FE23B
:1019B000C82E81E0D82E8A01AA24A394B12C25E058
:1019C000922EF3E3CF16F1E0DF0609F44AC0F601E8
:1019D00081916F01E82FE295EF70F0E021A18F7007
:1019E000A50102C0440F551F8A95E2F7CA01922F44
:1019F000982B91A392A18095892382A350EA5A95AE
:101A0000F1F7E6E4F1E020E040E050E03191A32F6F
:101A1000A295AF70B0E090968C9190E03F7002C0BC
:101A2000959587953A95E2F780FD07C0C501042E8C
:101A300001C0880F0A94EAF702C080E090E0282BEA
:101A40004F5F5F4F4730510509F7F80180818217DA
:101A500019F02083909200010E949C0C0F5F1F4F91
:101A6000B0CF809100018823B1F0815080930001B4
:101A7000811103C0C153DE4F07C08FE99FE001977A
:101A8000F1F700C0000007C0F70191917F01999321
:101A90008F5F8430C9F781E0DF91CF911F910F9163
:101AA000FF90EF90DF90CF90BF90AF909F90089500
:101AB000EF92FF920F931F93CF93DF938091DF01FB
:101AC000882309F47AC00E94BF0C8091040181111F
:101AD00003C0C4E0D0E002C0C0E0D0E0C153DE4F9C
:101AE00044E050E0BE018BEB91E00E94C92C7C01E8
:101AF00088819981AA81BB818093BB019093BC01AD
:101B0000A093BD01B093BE0180910401811103C077
:101B1000C0E0D0E002C0C4E0D0E09091020180912A
:101B20000101981761F082E090E00E94C92A8C01BF
:101B3000892B39F4809101018093020102C000E0F9
:101B400010E0EF2849F48091560190915701892BBC
:101B500019F480E090E002C081E090E00E94C92A80
:101B6000892B49F48091BF018093010110925701A4
:101B70001092560106C081E090E090935701809347
:101B800056010115110531F00230110509F050C060
:101B900028984EC0289AC153DE4F8091B60190918B
:101BA000B701A091B801B091B90188839983AA8344
:101BB000BB835D9A1092580152C00E94BF0C809165
:101BC0000401811103C0E4E0F0E002C0E0E0F0E0D5
:101BD000E153FE4F80E020E030E0D901AA54BE4F2F
:101BE0004C919191491381E09C932F5F3F4F24309A
:101BF000310599F79091BF01890F8093BF018091C2
:101C00000401811103C080E090E002C084E090E014
:101C1000FC01E153FE4F4091BB015091BC0160912A
:101C2000BD017091BE01408351836283738317C0ED
:101C30005D98809158018F5F80935801863078F0CD
:101C400080910401811103C0E0E0F0E002C0E4E013
:101C5000F0E0E153FE4F108211821282138281E084
:101C6000DF91CF911F910F91FF90EF9008950F9307
:101C70001F93CF93DF93C62FD42F122FFC018281A5
:101C80008823C9F06093B0010E94831C9093AB013C
:101C90008093AA0180E28C0F883008F057C0C7708B
:101CA00081E001C0880FCA95EAF7DF91CF911F91BB
:101CB0000F910C94C2258091B001681330C08091BF
:101CC000AA019091AB010E94591C8639910538F503
:101CD00000E20D0FCD17B9F080E28C0F883040F490
:101CE000C77081E001C0880FCA95EAF70E94B72546
:101CF000083028F581E09D2F977001C0880F9A95D4
:101D0000EAF70E94C225812F0E94CC250830F0F40A
:101D1000D77081E001C0880FDA95EAF70AC080E247
:101D20008C0F883098F4C77081E001C0880FCA9585
:101D3000EAF7DF91CF911F910F910C94B725812F76
:101D4000DF91CF911F910F910C94CC25DF91CF9112
:101D50001F910F9108950E94831C9093030280931A
:101D600002028091040281110BC062E070E088E100
:101D700093E00E94AC1F892B19F481E08093040248
:101D80008091040208956091DF04669570E041E05F
:101D900050E083E091E00E94BC2C892B19F481E093
:101DA000809320020E94831C90931A028093190250
:101DB00008959091DF0490FF36C09170811102C0A8
:101DC000926006C08F3010F09C6102C0880F982B83
:101DD0009093DF04662351F06091DF047091E0047A
:101DE0008091E1049091E2040E94D2096091DF04A5
:101DF000669570E041E050E083E091E00E94BC2CE9
:101E0000892B19F01092200202C00E94C30E81E0BB
:101E100080931C0220E04091E2046091E1048091F3
:101E2000E0040C94E40908958091DF0486958150C4
:101E300009F48EE061E00C94D90E8091DF04869560
:101E40008F5F8F3008F081E061E00C94D90E4F92E3
:101E50005F926F927F928F929F92AF92BF92CF923A
:101E6000DF92EF92FF920F931F93CF93DF9300D0F7
:101E700000D01F92CDB7DEB7FC010081D1808381F5
:101E80009481892B41F088248A94D81006C091E06F
:101E90000F3F19F403C091E001C090E090FDD3C55D
:101EA0007F0185E0DE01119601900D928A95E1F7A0
:101EB000F701228189819A81222349F00E94081E1C
:101EC000182F682F89819A810E94811E03C00E9469
:101ED000551E182F28E3129FF001112487E0D89E89
:101EE000E00DF11D1124E00FF11DEE0FFF1FE65E66
:101EF000FC4F05911491073F9CE5190789F4F70100
:101F00008281882309F458C00E94390A8091DF0435
:101F100081608093DF0461E086950E94D90E4CC0F9
:101F2000003FFCE51F07C9F180F4083D8CE5180768
:101F3000C9F0093D9CE51907E1F1073DECE51E07F5
:101F4000D9F526E241EE61EE10C0023FFCE51F0725
:101F500061F138F1033F8CE5180771F520E341E0AA
:101F600067EE03C027E245EE65EEC7010F900F90C4
:101F70000F900F900F90DF91CF911F910F91FF90D5
:101F8000EF90DF90CF90BF90AF909F908F907F9019
:101F90006F905F904F900C94370E23EE41E060EE0F
:101FA000E4CF28E241E064EEE0CF2FE241E062EED0
:101FB000DCCF28E241E0D8CFF7018281882309F401
:101FC0000DC31092B001093CFCE51F0709F408C4D9
:101FD000F0F5023C8CE5180709F479C3C0F405312B
:101FE000ECE51E0778F40230FCE51F0708F090C40A
:101FF00001152CE5120709F419C301301C4509F03D
:102000005BC045C306311C4509F056C0E8C4053C19
:10201000ECE51E0709F4CAC350F4033C2CE5120793
:1020200009F48EC3043C1C4509F046C0A4C3073C18
:102030009CE5190709F4C3C308F0C8C38091E00404
:1020400021E04091E2046091E1048A50DBC30F3C3F
:10205000FCE51F0709F43BC4C0F40C3C8CE51807F1
:1020600009F4EDC348F40A3CECE51E0709F4BFC3CC
:102070000B3C1C4509F5DDC30D3C2CE5120709F4AA
:1020800004C40E3C1C45C1F419C4063D9CE5190767
:1020900028F4013D1C4508F423C4D5C40D3DFCE5DE
:1020A0001F0709F429C40E3D2CE5120709F4F8C2F4
:1020B0000C3D1C4509F41DC4F70100811181C801C4
:1020C0000E94081ED82E682FC8010E94811EB801E8
:1020D0008D2D0E94490A182FD92E082FF701C5808F
:1020E000C2943FE0C322F280F11010926502ED2C01
:1020F000E2942FE0E2228E2D90E08C30910508F0E2
:1021000046C2FC01EA5AFF4F0C94B62C9D2D9F70DD
:102110008D2D807FB92E19F0B29490EFB922FF2057
:10212000C9F0BB2009F41FC280E2810F883010F093
:10213000011107C080916B02082F0B2900936B02DD
:1021400006C080916502082F0B29009365020E944A
:10215000E41D09C2812F0E948028BB2009F417C208
:102160009B2D909580E2810F883010F0011107C0FF
:1021700080916B02082F092300936B0206C08091A7
:102180006502082F0923009365020E94E41DFFC128
:102190008D2D8F709D2D907F903211F08295807FD4
:1021A000013069F4FF2029F0F2E0FC1508F4EFC1DA
:1021B0007BC1882483948C1408F4E9C17BC1FF207F
:1021C00021F0CC2009F470C1CEC1CC2009F472C139
:1021D000093309F0D9C1CFC18D2D869586958370BD
:1021E00019F0813061F0D3C1FF2021F0812F9D2DA6
:1021F000937002C080E090E00E94D908D3C1FF2014
:1022000021F0812F9D2D937002C080E090E00E940C
:10221000C308C8C1FF20F9F0053F51F0063F71F037
:10222000043FA9F48091B4019091B50181600BC085
:102230008091B4019091B501826005C08091B40194
:102240009091B50184609093B5018093B401812F82
:102250000E94CB1B1EC0053F51F0063F71F0043FAA
:10226000A9F48091B4019091B5018E7F0BC080914B
:10227000B4019091B5018D7F05C08091B40190911A
:10228000B5018B7F9093B5018093B401812F0E949B
:10229000011B0E948F1C86C18D2D837009F072C0B6
:1022A000F1107EC1912F929596959770990F990F85
:1022B000812F8F70882E912CA12CB12C24013501F7
:1022C000092E04C0440C551C661C771C0A94D2F7D6
:1022D00014FF12C04FE050E060E070E004C0440F13
:1022E000551F661F771F9A95D2F7DB01CA018095AB
:1022F0009095A095B09503C080E090E0DC012D2D75
:10230000269526952370223009F198F58090DB01FF
:102310009090DC01A090DD01B090DE01213059F0F9
:1023200084299529A629B729BC01CD0168217921E5
:102330008A219B2124C084289528A628B728BC017F
:10234000CD01682979298A299B2919C084299529D1
:10235000A629B7298090DB019090DC01A090DD01D7
:10236000B090DE01BC01CD01682579258A259B2529
:1023700006C0BC01CD0164297529862997290E94D0
:102380002F230EC1FF2019F08D2D817001C086957D
:10239000882309F405C1912F929596959770990F0E
:1023A000990F812F8F70882E912CA12CB12C240194
:1023B0003501092E04C0440C551C661C771C0A9478
:1023C000D2F714FF12C04FE050E060E070E004C0AC
:1023D000440F551F661F771F9A95D2F7DB01CA017C
:1023E00080959095A095B09503C080E090E0DC01C9
:1023F0002D2D269526952370223009F198F5809091
:10240000D7019090D801A090D901B090DA01213085
:1024100059F084299529A629B729BC01CD01682145
:1024200079218A219B2124C084289528A628B728B1
:10243000BC01CD01682979298A299B2919C08429E1
:102440009529A629B7298090D7019090D801A0900E
:10245000D901B090DA01BC01CD01682579258A2522
:102460009B2506C0BC01CD016429752986299729C1
:102470000E94F32295C0812F003FF9F018F4003E2E
:1024800050F46DC0023F09F44BC008F442C0033F52
:1024900009F44DC064C0012F0F708D2D8F71FF2086
:1024A00031F00E94D11E802F0E94C22570C00E9470
:1024B000AC1E802F0E94B7256AC0FF2021F1E1E009
:1024C000EC1508F464C02D2D2F7181E090E0A0E0A0
:1024D000B0E0AC01BD0104C0440F551F661F771F5B
:1024E0002A95D2F78091D7019091D801A091D90176
:1024F000B091DA014A015B0188269926AA26BB26FB
:10250000C501B40125C082E0982E9C1408F43FC098
:10251000DACFFF2039F08D2D8F710E94D11E37C088
:10252000FF20C9F38D2D8F710E94AC1E30C0FF209B
:1025300091F02D2D2F7181E090E0A0E0B0E0BC0182
:10254000CD0104C0660F771F881F991F2A95D2F707
:102550000E94F3221CC060E070E0CB01F9CFFF20A5
:1025600031F0CC20C1F2812F0E94B92810C0CC20BC
:10257000C9F2893349F42FEF87EE93E02150804070
:102580009040E1F700C00000812F0E948028E8E021
:10259000EE1631F0EE1630F086EF8E0D823010F42C
:1025A0000E94EF08812F9D2D0E94AB23811105C051
:1025B0001092B3011092B20146C2FF2019F0C1106F
:1025C000F7CF41C2C110F4CF8091B2019091B30115
:1025D000029771F7812F0E94CC25EACF013DFCE5DF
:1025E0001F07C0F4023C2CE5120708F02CC205318D
:1025F0008CE5180750F402309CE5190708F080C1FB
:1026000001151C4508F47CC11EC206311C4509F0A9
:1026100077C1F5C1063D2CE5120708F414C20C5D24
:102620001C450330110508F06BC10DC210926B02FE
:102630000E94A4258FEF94E3ECE081509040E040AD
:10264000E1F700C0000081E08093E00080E2809329
:10265000D8001092C9008FE19EE40197F1F700C005
:10266000000087E090EBDC018093E9049093EA049A
:10267000A093EB04B093EC049CE088E10FB6F894CF
:10268000A895809360000FBE90936000FFCF80916B
:102690001002982F909590FB80F980931002D3C17F
:1026A0000F900F900F900F900F90DF91CF911F918F
:1026B0000F91FF90EF90DF90CF90BF90AF909F90E1
:1026C0008F907F906F905F904F900C94361D80910B
:1026D000DF0480FF2FC08E7F8093DF046091DF04D2
:1026E0007091E0048091E1049091E2040E94D2098B
:1026F000109220029FEFE0E7F2E09150E040F040BE
:10270000E1F700C000000F900F900F900F900F9016
:10271000DF91CF911F910F91FF90EF90DF90CF90BD
:10272000BF90AF909F908F907F906F905F904F90F1
:102730000C94FB0881608093DF0461E08695A7C05C
:1027400080916B028272D9F00F900F900F900F90D2
:102750000F90DF91CF911F910F91FF90EF90DF903D
:10276000CF90BF90AF909F908F907F906F905F9031
:102770004F900C94140F80916B02827229F30F908A
:102780000F900F900F900F90DF91CF911F910F91AD
:10279000FF90EF90DF90CF90BF90AF909F908F9081
:1027A0007F906F905F904F900C941D0F8091E0048C
:1027B00021E04091E2046091E104865F23C06091D2
:1027C000E10420E1620F08F46FEF06C06091E104BC
:1027D00020E1621B08F460E021E04091E20410C0B7
:1027E0004091E20420E1420F08F44FEF06C040910F
:1027F000E20420E1421B08F440E021E06091E104A2
:102800008091E0040F900F900F900F900F90DF9148
:10281000CF911F910F91FF90EF90DF90CF90BF90DD
:10282000AF909F908F907F906F905F904F900C949F
:10283000E4098091E304833048F48F5F05C0809100
:10284000E304882319F081508093E3046091DF044E
:102850007091E0048091E1049091E2040F900F9058
:102860000F900F900F90DF91CF911F910F91FF90DC
:10287000EF90DF90CF90BF90AF909F908F907F9020
:102880006F905F904F900C94D20961E081E00F90BF
:102890000F900F900F900F90DF91CF911F910F919C
:1028A000FF90EF90DF90CF90BF90AF909F908F9070
:1028B0007F906F905F904F900C94D90E0E94B0095A
:1028C0008250833008F45BCF61E082E0E0CF0E9469
:1028D000B0098650823008F452CF61E086E0D7CF4D
:1028E0000E94B0098950853008F449CF61E089E041
:1028F000CECF1092DD04A7C082E08093DD04A3C098
:10290000F70100811181C8010E94551ED82EDFCB2E
:102910000E942B1D811102C00E94361D84E090E0B0
:102920000E943A2C90E09093CB018093CA01F80169
:10293000E350FC45E231F10530F4EE59FF4F809150
:10294000CA010C94B62C8091CA01816027C08260B4
:1029500025C0846023C0806121C080621FC0806464
:102960001DC080681BC08460886018C08E7F16C040
:102970008D7F14C08B7F12C08F7E10C08F7D0EC0E4
:102980008F7B0CC08F770AC08B7F877F07C087FB48
:10299000222720F991E0922790FB87F98093CA01C2
:1029A0006091CA0184E090E00E944E2C10926B026C
:1029B0000F900F900F900F900F90DF91CF911F917C
:1029C0000F91FF90EF90DF90CF90BF90AF909F90CE
:1029D0008F907F906F905F904F900C94A425809182
:1029E0006B028A7A91E009F490E09093B101811131
:1029F00026C069E281E292E00E94F61C09C0809143
:102A0000B10181111EC069E281E292E00E94CE1CF8
:102A10000F900F900F900F900F90DF91CF911F911B
:102A20000F91FF90EF90DF90CF90BF90AF909F906D
:102A30008F907F906F905F904F900C94E41D65E3B2
:102A4000D9CF65E3E1CF0F900F900F900F900F90CB
:102A5000DF91CF911F910F91FF90EF90DF90CF907A
:102A6000BF90AF909F908F907F906F905F904F90AE
:102A70000895CF93DF9300D01F92CDB7DEB720919A
:102A80009002243031F523E02983805891099B83FB
:102A90008A8382E08093E9008FEF9091E800815073
:102AA00095FD06C095ED9A95F1F700008111F5CFDF
:102AB0008091E80085FF0DC040E050E063E070E0E9
:102AC000CE0101960E94D51F8091E8008E778093F9
:102AD000E8000F900F900F90DF91CF9108950F9322
:102AE0001F93CF93DF9300D01F92CDB7DEB78C0139
:102AF0000E947428823011F0843021F584E08983AB
:102B00001B830A8382E08093E9008FEF9091E800B5
:102B1000815095FD06C095ED9A95F1F70000811161
:102B2000F5CF8091E80085FF0DC040E050E063E004
:102B300070E0CE0101960E94D51F8091E8008E774B
:102B40008093E8000F900F900F90DF91CF911F912D
:102B50000F910895CF93DF93CDB7DEB72C970FB6C3
:102B6000F894DEBF0FBECDBF84B7877F84BF0FB69A
:102B7000F894A8958091600088618093600010921D
:102B800060000FBE80E8809361001092610085B7FD
:102B9000806885BF85B7806885BF8EE090E00E9421
:102BA0003A2C91E0811101C090E090930401809152
:102BB000D80080618093D8000AE10A95F1F700C03F
:102BC0008091D90063E070E080FF05C085E091E06E
:102BD0000E94E72904C085E091E00E94F0297894E2
:102BE0000E9423260E94C9268091E200846080937F
:102BF000E2007894809190028823A1F01091E9007E
:102C00001F709091EC00892F817090FD80E8182B47
:102C10001092E9008091E80083FD0E9401201F705E
:102C20001093E90082E084BD93E095BD9AEF97BDD3
:102C300080936E0080911002836088608093100200
:102C40000E949C0CA6E4B1E04DE451E061E070E02C
:102C50008D91E82FE295EF70F0E021A18F708B014C
:102C600002C0000F111F8A95E2F7C801902F9095BE
:102C7000922391A392A1892B82A34A175B0741F764
:102C8000559A209A5D9A289AA1ECB1E017EDA12EF1
:102C900011E0B12EEFECF1E011921D92AE16BF06DD
:102CA000D9F78091D80080618093D8001AE11A95F5
:102CB000F1F700C08091D90081708093DF010E94FC
:102CC0002B1D811102C00E94361D8091DF018111F0
:102CD00002C082E001C083E08093000280FD02C058
:102CE00080E801C080E280939A020E944C2B6DE044
:102CF00070E08DE396E00E94AC1F892B99F58091DE
:102D0000000263E070E081FD2AC08AE396E00E9441
:102D1000AC1F892B39F56DE070E08AE296E00E94E5
:102D2000AC1F892BF9F4EDE9F2E080E092E0DF01DD
:102D30008C011D9201501040E1F7F093A404E09340
:102D4000A3048FEF9FEF90939C0280939B0281E0FE
:102D500080930502809304021092010203C087E36E
:102D600096E0D5CF0E942B1D811102C00E94361D16
:102D700082E090E00E943A2C8093100284E090E080
:102D80000E943A2C90E09093CB018093CA0183E09B
:102D900090E00E943A2C682F70E080E090E00E9462
:102DA0002F238091C901811138C080911002816068
:102DB000809310020E942B1D811104C00E94361DB9
:102DC0000E94390A88E090E00E94422C6093DF0460
:102DD0007093E0048093E1049093E2046E7F71F4B9
:102DE0000E94390A88E090E00E94422C6093DF0440
:102DF0007093E0048093E1049093E2040E94B80988
:102E0000109220028091DF0480FF04C060E086956C
:102E10000E94D90E81E08093C9018091CA01806827
:102E20008093CA0184E291E09093CD018093CC011C
:102E3000CC24C394D12C80919002853009F056C0E7
:102E400080919002843009F441C01092CE0120E4B8
:102E500088E190E00FB6F894A895809360000FBECB
:102E600020936000109220028091E504811117C028
:102E700081E08093E5048091DF04982F9170909316
:102E8000E4048E7F8093DF041FEF20E732E01150CF
:102E900020403040E1F700C000000E94FB0883B7EB
:102EA000817F846083BF83B7816083BF7894889576
:102EB00083B78E7F83BF0FB6F894A895809160008A
:102EC000886180936000109260000FBE80918F0235
:102ED000882309F4B0CF0E94580DEFECF1E0819106
:102EE000811100C3AE16BF06D1F7A5CF0E94580DC1
:102EF000982EA1E1B2E0EFECF1E0E12CF12C7E2D77
:102F000061912D912627B1F180E090E030E0182FFB
:102F1000A901082E02C0559547950A94E2F740FF93
:102F200025C089837A83C60102C0880F991F1A952C
:102F3000E2F78C01862F90E08023912321E0892BFA
:102F400009F420E02B830E94831C8160782F9D83ED
:102F50008C8349815A816B818D810E940808F70119
:102F6000EF5EFD4F8081082700831CC001968730EB
:102F7000910569F69FEFE91AF90A08E0E016F104F5
:102F800009F0BDCF8FEF8E838F8318860E94831C3C
:102F90008160782F9A8789874E815F8168858A85CD
:102FA0000E94080880910502882309F49EC12DE93A
:102FB00032E03093A4042093A3048091DF0188239E
:102FC00009F497C06091DB017091DC018091DD0113
:102FD0009091DE010E94941D882329F0813039F4FC
:102FE00085ED96E002C08BED96E00E949E1F83ED7A
:102FF00096E00E949E1F6091D7017091D801809148
:10300000D9019091DA010E94941D833099F038F42F
:10301000882369F08230B9F485EB96E016C08530DC
:1030200079F058F0863079F48FEA96E00EC08DEC96
:1030300096E00BC087EC96E008C081EC96E005C0F6
:103040008BEB96E002C089EA96E00E949E1F87EA19
:1030500096E00E949E1F10916B02812F817119F4DE
:103060008BE996E002C081EA96E00E949E1F812FC4
:10307000827219F48FE896E002C085E996E00E941A
:103080009E1F812F847419F483E896E002C089E8BA
:1030900096E00E949E1F187819F48EE696E002C012
:1030A00084E796E00E949E1F81E896E00E949E1FA2
:1030B0000E94EF08182F8AE796E00E949E1F10FDDD
:1030C00003C082E696E002C088E696E00E949E1F5A
:1030D00011FD03C086E596E002C08CE596E00E94F3
:1030E0009E1F12FD03C08AE496E005C080E596E0CD
:1030F00002C081EE96E00E949E1F20919B023091BB
:103100009C022115310509F4D9C080910102811179
:10311000D5C0282E312C7601082E02C0EE0CFF1CE3
:103120000A94E2F7A70142235323452B11F48F5F42
:10313000F0CF909100029101E5E0220F331FEA9554
:10314000E1F790FD12C08295880F807680931F0171
:10315000220F232F221F330B319520932201815EF2
:10316000809320011092230112C065E036952795C7
:103170006A95E1F7220F220F220F20931F01109270
:103180002201295F2093200183E08093230124E61C
:1031900030E047E050E06DE171E088E70E94D92B14
:1031A000892B09F08BC08091000280FD23C0C101F2
:1031B00055E0880F991F5A95E1F7AC0143565D4FD2
:1031C00004E610E020E230E060E488E70E94002C92
:1031D000892B09F073C00E94AB0EE094F0948091AB
:1031E0009B0290919C02E822F922F0929C02E092CC
:1031F0009B0264C080E2A0EEB1E01D928A95E9F7DF
:1032000045E0220C331C4A95E1F7E1E5F1E0FC874B
:10321000EB874DE451E0AB85BC858D91BC87AB87D6
:10322000FA019191AF019101290F311D89010356D6
:103230001D4F280190E080529E4FFC0107E09F0146
:10324000281B390B7C2C01C0770C2A95EAF7B201B8
:10325000812CDB011D91BD011721202F281927701A
:10326000622E022E000C330BB12F01C0BB0F6A94EB
:10327000EAF76B2E3195219531092770332701C06C
:1032800016952A95EAF7612A1081612A6082839453
:1032900018E08112DECF015031960F3F81F625E50F
:1032A00031E06B857C852617370709F0B4CF04E63B
:1032B00010E020E230E040EE51E086CF8091040241
:1032C000882399F080910202909103020E94591C78
:1032D00081369A4E50F062E070E081E297E00E9401
:1032E000AC1F892B11F41092040291100E94AB0EB6
:1032F00080910D0290910E020E94591C9C019091A8
:103300000C02992321F02031310508F478C0809116
:1033100008021091090281110BC01111F9C020910E
:103320000A022111F5C020910B022111F1C067C0E2
:103330009F3F19F09F5F90930C02181624F40E948F
:10334000A61B809308028091080287FF05C00E9497
:10335000A61B819580930802111624F40E94A61BD7
:10336000809309028091090287FF05C00E94A61B75
:10337000819580930902309108023323E1F0209176
:1033800009022223C1F005EB3003C0011124992367
:1033900019F09093080203C081E08093080215EBB6
:1033A0002103C0011124992319F09093090203C04D
:1033B00081E08093090280910A02181624F40E9489
:1033C000861B80930A0280910A0287FF05C00E9433
:1033D000861B819580930A0280910B02181624F4B3
:1033E0000E94861B80930B0280910B0287FF05C011
:1033F0000E94861B819580930B020E948F1C0E9465
:10340000EF0890910F02891721F00E94EF08809336
:103410000F0280912002882309F40DCD80911F02B4
:10342000E091DF04E695E81BE0931B02823059F43B
:10343000F0E0E75DF84FE4910E2F10E03CE9E32E59
:1034400039E0F32E21C0863059F4F0E0EA5DF84F00
:10345000E4910E2F10E02CE8E22E29E0F22E14C0A9
:10346000893061F4E695F0E0ED5DF84FE4910E2FC0
:1034700010E091E3E92E99E0F92E06C000ED17E087
:1034800084E4E82E87E0F82E80911C02882389F0DE
:1034900010921C020E94831C980120953095820F87
:1034A000931F90931A028093190210921E02109299
:1034B0001D028091190290911A020E94591C8017D6
:1034C000910708F4B8CCE0911902F0911A020E0F9E
:1034D0001F1F10931A020093190289E192E0F7016D
:1034E0000995A9CC80E189BD82E189BD09B400FEBE
:1034F000FDCF8091D8008F7D8093D8008091E0002F
:1035000082608093E0008091E00081FDFCCF93CC4D
:103510009F3F09F00FCF20CF80916D020895CF9388
:10352000DF93EC010E947428823011F08430F9F4AA
:1035300082E08093E9008FEF9091E800815095FD43
:1035400006C095ED9A95F1F700008111F5CF8091B5
:10355000E80085FF0CC040E050E066E070E0CE017E
:103560000E94D51F8091E8008E778093E800DF915C
:10357000CF910895CF93DF93EC010E94742882309D
:1035800011F08430D9F580912E01882339F0809193
:10359000CA0187FF03C060E282E002C068E081E008
:1035A0008093E9008FEF9091E800815095FD06C06F
:1035B00095ED9A95F1F700008111F5CF8091E80023
:1035C00085FF1CC080912E01811105C040E050E0B4
:1035D00068E070E003C070E040E050E0CE010E947F
:1035E000D51F8091E8008E778093E80080E2FE018D
:1035F000AEE6B2E001900D928A95E1F7DF91CF91AE
:103600000895803F39F48091090287FF6CC01092C1
:10361000090269C0813F29F4809109021816BCF3A0
:1036200062C090910802823F29F497FF5CC010921B
:10363000080259C0833F19F41916CCF354C0893FCE
:1036400041F480910A0218160CF04DC010920A0243
:103650004AC08A3F29F480910A0287FF44C0F6CF0E
:103660008B3F39F480910B0287FF3DC010920B0213
:103670003AC08C3F29F480910B021816BCF333C07A
:10368000843F21F4809107028E7F17C0853F21F48B
:10369000809107028D7F11C0863F21F4809107023F
:1036A0008B7F0BC0873F21F480910702877F05C085
:1036B000883F31F4809107028F7E8093070213C008
:1036C0008D3F21F480916A028E7F0BC08E3F21F4E2
:1036D00080916A028D7F05C08F3F29F480916A0234
:1036E0008B7F80936A028091080281110EC08091C5
:1036F000090281110AC080910A02811106C08091DD
:103700000B02811102C010920C02089580916A028E
:1037100080FD18C081FD14C082FD16C080910C028E
:10372000882381F0883280F424E0829FC001112434
:1037300068E270E00E94A22C862F672B19F005C06A
:1037400082E0089581E0089584E0089580916A02FE
:1037500080FD18C081FD18C082FD18C020910C02A8
:103760002223B1F08EE12032A8F4289F9001112489
:1037700085E0359527958A95E1F7822F232B51F423
:1037800081E0089587E008958FE008958EE108951F
:1037900085E008950895803F21F40E94A61B81953D
:1037A00004C0813F29F40E94A61B8093090208955A
:1037B000823F21F40E94A61B819504C0833F29F417
:1037C0000E94A61B809308020895893F19F40E9465
:1037D000861B05C08A3F31F40E94861B8195809329
:1037E0000A0208958B3F21F40E94861B819504C034
:1037F0008C3F29F40E94861B80930B020895843F1E
:1038000021F480910702816017C0853F21F48091E7
:103810000702826011C0863F21F480910702846014
:103820000BC0873F21F480910702886005C0883F64
:1038300031F48091070280618093070208958D3FE3
:1038400021F480916A0281600BC08E3F21F4809147
:103850006A02826005C08F3F29F480916A02846009
:1038600080936A02089578941F920F920FB60F9278
:1038700011248F939F93AF93BF9380916602909191
:103880006702A0916802B09169020196A11DB11D65
:103890008093660290936702A0936802B0936902D6
:1038A000BF91AF919F918F910F900FBE0F901F907E
:1038B0001895CF92DF92EF92FF920F931F932FB73D
:1038C000F89440916602509167026091680270918D
:1038D00069022FBF6A017B01EE24FF248C0120E0E6
:1038E00030E0C016D106E206F30610F4415051094B
:1038F0009A01281B390BC9011F910F91FF90EF907E
:10390000DF90CF9008952FB7F89480916602909140
:103910006702A0916802B09169022FBF0895E091FB
:10392000CC01F091CD01309749F082E080930602FE
:103930000480F581E02D86E092E009950E94831CC9
:1039400090930E0280930D0208951F920F920FB66E
:103950000F9211248F939F93AF93BF938091CE01C9
:10396000811113C08091660290916702A091680254
:10397000B09169024196A11DB11D8093660290939A
:103980006702A0936802B0936902BF91AF919F91C3
:103990008F910F900FBE0F901F90189520912E01C0
:1039A0002223C9F02091CA0127FF15C0262F269592
:1039B000269526952E31C8F4FC01E20FF11D6770A3
:1039C00081E090E001C0880F6A95EAF780959281C6
:1039D000892382830895FC0106962281621301C027
:1039E00012823196E817F907C1F7089520912E0148
:1039F0002223C1F02091CA0127FF14C0262F26954B
:103A0000269526952E3130F5FC01E20FF11D6770E9
:103A100081E090E001C0880F6A95EAF79281892BD6
:103A200082830895FC0132962FEF30E041916417B4
:103A300089F02F3F19F4411101C0232F3F5F363029
:103A4000A9F72F3F39F0FC01E20FF11D27FDFA9590
:103A500062830895089580E090E00E94482C21E060
:103A60008D3E9E4F09F020E0822F08956DEE7EEF8F
:103A700080E090E00E946C2C60E082E090E00E9488
:103A80004E2C60E083E090E00E944E2C1092DB010F
:103A90001092DC011092DD011092DE0160E084E002
:103AA00090E00E944E2C60E085E090E00E944E2C59
:103AB00060E086E090E00E944E2C6FEF87E090E09F
:103AC0000E944E2C40E050E0BA0188E090E00E9455
:103AD000602C60E08DE090E00E944E2C40E050E0D1
:103AE000BA0188E190E00E94602C60E087E190E0FC
:103AF0000E944E2C40E050E0BA018CE190E00E9420
:103B0000602C60E080E290E00E944E2C40E050E0AB
:103B1000BA018FE090E00E94602C40E050E0BA01D2
:103B200083E190E00C94602CCF92DF92EF92FF92B1
:103B30006C01EE24FF24C114D104E104F10421F04E
:103B4000C701B60120E101C020E0C72ED82EE92E22
:103B5000FF24C114D104E104F10419F0285FC70166
:103B6000B6016B017C0154E0F694E794D794C794B6
:103B70005A95D1F7C114D104E104F10419F02C5F76
:103B8000C701B6016B017C0142E0F694E794D7943B
:103B9000C7944A95D1F7C114D104E104F10419F096
:103BA0002E5FC701B601DC01CB01B695A7959795AD
:103BB0008795892B8A2B8B2B09F02F5F822FFF9003
:103BC000EF90DF90CF90089590916B028091650205
:103BD000892B90916402892B80932102E091CC0182
:103BE000F091CD01309799F090912E01992349F0F1
:103BF0009091CA0197FF05C08093220285E08093CF
:103C000021020280F381E02D81E292E0099408957F
:103C1000BF92CF92DF92EF92FF920F931F93CF93B9
:103C2000DF938C01C090D701D090D801E090D901EA
:103C3000F090DA018091DB019091DC01A091DD012F
:103C4000B091DE01C82AD92AEA2AFB2ACFE1D0E0C6
:103C5000D701C6010C2E04C0B695A79597958795F8
:103C60000A94D2F780FD04C0219790F7B12C07C0C9
:103C7000BC2EB8018C2F0E94490A0197A9F38B2D05
:103C8000DF91CF911F910F91FF90EF90DF90CF9038
:103C9000BF900895CF93DF93EC010E94081EBE01F0
:103CA0000E94490ADF91CF91089527E0929F800DED
:103CB0001124682F669566956695982F977085E014
:103CC000689FB001112440E050E080E0FB01E40F68
:103CD000F51FEF5BFD4F208130E0092E02C03695C5
:103CE00027950A94E2F721703327042E01C0220F92
:103CF0000A94EAF7822B4F5F5F4F4530510531F749
:103D0000089527E0929F800D1124E82FE695E6950F
:103D1000E695877051E001C0550F8A95EAF785E076
:103D2000E89FF0011124EF5BFD4F20E030E070E0F0
:103D30004081CB01022E02C0969587950A94E2F746
:103D40008170819584278523842781932F5F3F4F3E
:103D50002530310569F708950F931F9341E050E036
:103D600060E070E004C0440F551F661F771F8A95FE
:103D7000D2F740955095609570958091D7019091BC
:103D8000D801A091D901B091DA018A019B010823E1
:103D900019232A233B23C901B8011F910F910C94C9
:103DA000F3220F931F9341E050E060E070E004C005
:103DB000440F551F661F771F8A95D2F78091D70150
:103DC0009091D801A091D901B091DA018A019B01AB
:103DD000082B192B2A2B3B2BC901B8011F910F91DE
:103DE0000C94F322CF93DF93C091A304D091A40449
:103DF0008A30B1F420919A02CE018D599240622FFF
:103E000070E00E948E2C281B822F66E00E94822C7C
:103E1000C82FC15008F48FC080E20E94F21EF9CF73
:103E20008D30E9F4CD59D24020919A02622F70E092
:103E3000CE010E948E2C281B822F9E01280F311D3F
:103E40002115324018F080E0C0E0D0E0C80FD11D4D
:103E5000C356DD4FD093A404C093A3046CC096E076
:103E6000FE01ADE9B4E001900D929A95E1F7813E33
:103E700030F086E0FE0111928A95E9F70BC0F6E07A
:103E80008F9FB00111246A54774F46E050E0CE0175
:103E90000E94312CC091A304D091A40446E050E0CC
:103EA000BE018DE994E00E94C92C892B49F19E0145
:103EB0002D593240A90185E0569547958A95E1F73D
:103EC00081E090E0BC0102C0660F771F4A95E2F7DF
:103ED00040919B0250919C02462B572B2A5F3F4FEB
:103EE00065E0369527956A95E1F702C0880F991F1E
:103EF0002A95E2F7842B952B90939C0280939B024A
:103F00009E012759324040919A02642F70E0C90106
:103F10000E948E2C481B463010F4240F311D2115B1
:103F200082E0380710F020E030E023563D4F309318
:103F3000A4042093A304DF91CF910895CF93DF933E
:103F4000EC01FE018491882321F00E94F21E21964B
:103F5000F8CFDF91CF910895EF92FF920F931F93C7
:103F6000CF93DF93EC017B0164E670E088E70E9469
:103F7000522B8C01EC0EFD1ECE15DF0561F017FDF6
:103F80000AC0FE01849164E670E00E94A92B8C01B6
:103F90002196892B89F30E942D2CC801DF91CF91A6
:103FA0001F910F91FF90EF900895EF92FF920F9362
:103FB0001F93CF93DF937C018B010E9442268111D6
:103FC00019C0E70101151105A1F08091E80085FDF8
:103FD0000AC08091E8008E778093E8000E94422614
:103FE000882381F307C089918093F1000150110962
:103FF000E9CF80E0DF91CF911F910F91FF90EF907B
:1040000008951F93CF93DF93CDB7DEB7AA970FB66E
:10401000F894DEBF0FBECDBFE2E9F2E08091F1007F
:10402000819322E0EA39F207C9F780919302833045
:1040300009F460C030F4813071F0823009F49CC022
:10404000B3C08A3009F488C08B3009F46BC0893062
:1040500009F0AAC020C080919202813A09F0A4C060
:104060008091E800877F8093E8008091960290918C
:104070009702892B21F460E28EE692E003C060E0B3
:1040800080E090E070E00E9416288091E8008B7735
:104090008093E80089C080919202813209F084C047
:1040A0008091960290919702029708F07DC08091CE
:1040B000E800877F8093E8008091E80082FD05C0DA
:1040C000809190028111F8CF6FC02091F300809110
:1040D000F20090E0922B029729F48091F1008B7FFF
:1040E000813021F48091F10080936D028091E8008D
:1040F0008B7756C080919202813A09F055C0809129
:10410000960290919702892B09F04EC08091E800A9
:10411000877F8093E8008091E80080FFFCCF80914A
:104120002E0139C0809192028132F1F58091960280
:1041300090919702892BC1F58091E800877F809349
:10414000E8000E9475268091940280932E011092BF
:104150006B020E94A42528C080919202813221F531
:104160008091E800877F8093E8000E947526809107
:10417000950280936C0218C080919202813AA1F45A
:104180008091E800877F8093E8008091E80080FFBD
:10419000FCCF80916C028093F1008091E8008E77D3
:1041A0008093E8000E9475268091E80083FFD8C1C3
:1041B0008091920290919302492F50E04A3051052C
:1041C00008F0CEC1FA01EC58FF4F0C94B62C8038A1
:1041D00021F0823809F0C4C108C080918E0290910C
:1041E0008F02992389F082600FC0809196028F70B0
:1041F000873008F0B5C18093E9008091EB0085FB22
:10420000882780F91092E9009091E800977F9093B9
:10421000E8008093F1001092F10071C1282F2D7FEA
:1042200009F09EC1882319F0823061F099C1809114
:104230009402813009F094C1933009F080E08093BA
:104240008F022EC08091940281112AC08091960223
:104250008F702FEF280F263008F082C18093E9007D
:104260002091EB0020FF1CC0933021F48091EB00E3
:10427000806214C09091EB0090619093EB0021E07C
:1042800030E0A90102C0440F551F8A95E2F7409320
:10429000EA001092EA008091EB0088608093EB00C6
:1042A0001092E9008091E800877F2CC1811158C1EC
:1042B000109194021F778091E3008078812B809386
:1042C000E3008091E800877F8093E8000E947526D4
:1042D0008091E80080FFFCCF8091E30080688093AC
:1042E000E300111102C082E001C083E080939002DC
:1042F00037C18058823008F033C180919402909188
:1043000095028C3D53E0950779F583E08A838AE234
:1043100089834FB7F894DE01139620E03EE051E226
:10432000E32FF0E050935700E49120FF03C0E295A3
:10433000EF703F5FEF708E2F90E0EA3010F0C7967D
:1043400001C0C0968D939D932F5F243149F74FBFD5
:104350008091E800877F8093E8006AE270E0CE01F8
:1043600001960E941628BAC0409196025091970279
:10437000292F332723303105B1F068F4213031057E
:1043800009F4FDC02230310509F0EAC08BE390E06A
:10439000EDE2F8E050C02132310581F122323105E1
:1043A00009F439C0DDC0992781309105B9F070F06A
:1043B00082309105D9F0039709F0D2C0EAE7F8E01E
:1043C000E4918E2F90E0EAE7F8E032C0E2EBF8E00B
:1043D000E4918E2F90E0E2EBF8E02AC0E0EAF8E00A
:1043E000E4918E2F90E0E0EAF8E022C0E0E8F8E007
:1043F000E4918E2F90E0E0E8F8E01AC041155105F5
:1044000009F4C2C04130510509F0AAC089E090E02A
:10441000E8E5F8E010C04115510509F4BAC0413093
:10442000510509F09DC080EC90E0EDE2F7E003C09B
:10443000009709F495C02091E800277F2093E800B9
:1044400020919802309199028217930708F49C01F9
:1044500040E02115310589F180919002882309F40B
:104460003DC08530D9F18091E80083FD37C080914F
:10447000E80082FD2FC08091E80080FFEACF4091E4
:10448000F3008091F20090E0942B2115310559F052
:104490008830910540F444914093F10031962150C9
:1044A00031090196F2CF41E0089709F040E0809190
:1044B000E8008E778093E800CCCF4111CDCF0AC0C1
:1044C00080919002882351F0853041F08091E8007E
:1044D00083FD04C08091E80082FFF2CF8091E80064
:1044E0008B778093E8003CC08038D1F58091E8005C
:1044F000877F8093E800809191028093F100809102
:10450000E8008E778093E8000E94752629C081110B
:1045100027C080919402909195029927029704F503
:104520008091E800877F8093E800109194021093B7
:1045300091020E947526111106C08091E30087FD4B
:1045400002C081E001C084E08093900242E061EC0F
:1045500081E00E94942642E261EC82E00E9494266F
:104560008091E80083FF1AC08091E800877F8093E4
:10457000E8008091EB0080628093EB000FC082E145
:1045800090E0E8E6F8E057CF89E090E0EFE3F8E06C
:1045900052CF80E490E0EDEEF7E04DCFAA960FB653
:1045A000F894DEBF0FBECDBFDF91CF911F9108956C
:1045B00010926502109264020E94E41DE6E0F2E0AF
:1045C00086E0DF011D928A95E9F710920C021092A5
:1045D0006A020E948F1C80E090E00E94D90880E06F
:1045E00090E00C94C308CF92DF92EF92FF926B01A0
:1045F0007C016091DB017091DC018091DD01909183
:10460000DE010E94941D882319F0813071F019C0D9
:10461000D701C60180739927AA27BB27C097A10598
:10462000B10569F46894C6F80CC0D701C60184725C
:104630009927AA27BB278497A105B10599F3E89488
:10464000C6F8C092D701D092D801E092D901F09279
:10465000DA01FF90EF90DF90CF900C94D822609316
:10466000DB017093DC018093DD019093DE010C94FB
:10467000D8228091DC049091AB04891719F08F5FE8
:104680008770FBCF0895CF938091AA0482958F7095
:1046900009F05FC08091A704882309F45AC0809173
:1046A000DC04B091AB047091A504A091A6044091E4
:1046B000A8045091A90491E07F3F09F090E0692F90
:1046C000C6E08B1709F445C04115510521F0AF3FF5
:1046D00021F020E003C021E001C0262F90E020FD62
:1046E00035C0C89FF001C99FF00D1124E455FB4F60
:1046F00021812A132BC02081271328C02281211158
:1047000025C0238134812417350710F42150310945
:10471000241B350B26393105C8F42091AA042F70CB
:1047200020612093AA0426E0289FF001299FF00D24
:104730001124EF54FB4F80818F708061808385EA64
:1047400094E00E94270FCF910C9439230196877033
:10475000B8CFCF910895E92FE295EF704E2F50E03A
:10476000FA013297EE30F105B0F4E258FF4F0C94A5
:10477000B62C803F91F018F4883E68F40EC0843F58
:1047800051F40BC0883E48F0813F29F406C093FBEA
:10479000882780F9089580E0089581E008950E94B7
:1047A0004A1E0E94AB230895AF92BF92CF92DF9230
:1047B000EF92FF920F931F93CF93DF93CDB7DEB7A6
:1047C00061970FB6F894DEBF0FBECDBF8C0185E0B8
:1047D000F801DE011D9601900D928A95E1F7D8014E
:1047E0003C9111962C9111971296EC905091A50442
:1047F0006091A6048091A8049091A904009731F0DB
:104800006F3F31F441E05F3F19F403C041E001C064
:1048100040E0B42FB170BB2E40FD43C1F801C3800E
:10482000D480A090A704AA2009F4E2C04091AA0471
:10483000C816D90628F0D601A81BB90BCD0104C0B3
:10484000809590958C0D9D1DFF24F39486399105DC
:1048500048F0F12C407F09F090C085EA94E00E9476
:10486000270F17C1842F807F09F052C0621312C036
:10487000531310C0FE2CE1100DC04F7040614093E7
:10488000AA0485EA94E00E94270F8091AA04F80107
:10489000858348C1CD2831F02F3F31F481E03F3F7F
:1048A00019F403C081E001C080E080FD03C081E015
:1048B0008E2502C080E090E0F82FF170FF2E80FF7F
:1048C0001CC08091DC044091AB0456E0841709F4CD
:1048D00006C190E0589FF001599FF00D1124E45556
:1048E000FB4F6181261306C06081361303C06281CD
:1048F000E61203C001968770E9CFFE2CEE2009F482
:1049000011C18091AA0481608093AA04F12C0AC18C
:10491000621308C0531306C0E11004C08091AA04BA
:10492000F80199C03D872E878D859E850E94CF23F3
:10493000882369F1EE2059F12091AA04822F8295F3
:104940008F7090E0029774F08091A5049091A60476
:1049500098878F831986DB86CA862C87CE010796B7
:104960000E94270F86E0F801A5EAB4E001900D92BD
:104970008A95E1F70E9443230DC0621771F03D87CD
:104980002E878D859E850E94CF2381111AC0C80174
:104990000E94270FFF24F394C5C05313F0CFE110FA
:1049A000EECF8091AA04F8018583C8010E94270FE9
:1049B00086E0E5EAF4E0DF011D928A95E9F7FA2C3A
:1049C000B1C0EE2021F32091AA04822F82958F702E
:1049D00090E002973CF28091A5049091A6049A83FE
:1049E00089831B82DD82CC822E83CE010196B8CFD3
:1049F000C816D90638F0C81AD90AB6E9CB16D104B8
:104A000050F007C0809590958C0D9D1D86399105BD
:104A100010F0F12C3EC0FE2CEE2009F4B8CF62134A
:104A200027C0531325C02091AA0420FD18C0822F4F
:104A300082958F70482F50E04115510581F0F801A3
:104A400025834F30510541F08F5F982F9295907FCD
:104A5000822F8F70892B8583C8010E94270F86E0E3
:104A6000F801A5EAB4E001900D928A95E1F75AC0E9
:104A70003D872E878D859E850E94CF23811172CF21
:104A80008091AA0481608093AA04C8010E94270F24
:104A900049C0E5EAF4E086E0DF011D928A95E9F776
:104AA00041C0EE2009F473CF3D872E878D859E850A
:104AB0000E94CF23F82E882309F469CF86E0F801FD
:104AC000A5EAB4E001900D928A95E1F78091A504E2
:104AD0009091A6040E944A1E0E94432323C03D8752
:104AE0002E878D859E850E944A1E292F22952F7024
:104AF000223028F49F7039F0811105C00BC024309A
:104B000028F49F7049F4805E883020F0C8010E942C
:104B1000270FBF2CFB2C06C0D80115969C91907FC7
:104B200091F7F8CF8F2D61960FB6F894DEBF0FBEC8
:104B3000CDBFDF91CF911F910F91FF90EF90DF904C
:104B4000CF90BF90AF90089580912E01882331F0CF
:104B50008091CA0187FF02C08EE101C086E0E3E2D6
:104B6000F2E0DF011D928A95E9F70C94D8228823A0
:104B700041F0809590916B02892380936B020C9495
:104B8000E41D0895882339F090916B02892B80935E
:104B90006B020C94E41D0895CF93C82F0E94B9288E
:104BA000C93349F42FEF87EE93E0215080409040C5
:104BB000E1F700C000008C2FCF910C9480281F9249
:104BC0000F920FB60F9211242F933F934F935F9341
:104BD0006F937F938F939F93AF93BF93CF93DF9305
:104BE000EF93FF93C091E900CF708091EC00D82F34
:104BF000D17080FDD0E81092E9008091F000877FAD
:104C00008093F00078940E9401201092E900809136
:104C1000F00088608093F000CD2BCF70C093E90046
:104C2000FF91EF91DF91CF91BF91AF919F918F91C4
:104C30007F916F915F914F913F912F910F900FBE98
:104C40000F901F901895E8EDF0E080818E7F8083B3
:104C50001092E2001092DA001092E100A0EEB0E0B3
:104C60008C9181608C9380818F77808319BCA7EDB4
:104C7000B0E08C918E7F8C9380818F7E80831092A8
:104C8000DE0408952091E4003091E50095E640911E
:104C9000EC00842F817040FF23C08091E80080FDEC
:104CA0001DC080919002882399F0853099F0809101
:104CB000EB0085FD11C04091E4005091E500241700
:104CC000350729F3915011F09A01E1CF84E008955E
:104CD00082E0089583E0089581E0089580E00895DA
:104CE0004091E80042FFDDCF08958091920287FF56
:104CF00011C08091E80082FD05C080919002811171
:104D0000F8CF11C08091E8008B770BC080919002A2
:104D1000882349F08091E80080FFF8CF8091E80077
:104D20008E778093E8000895982F973068F59093D8
:104D3000E900981739F07091EC002091ED00509146
:104D4000F00003C0242F762F50E021FD02C09F5FAA
:104D5000ECCF3091EB003E7F3093EB003091ED00D3
:104D60003D7F3093ED003091EB0031603093EB00EC
:104D70007093EC002093ED005093F0002091EE0032
:104D800027FDE5CF80E008958F708093E90081E0F2
:104D90000895CF92DF92EF92FF920F931F93CF93DC
:104DA000DF93C8EDD0E088818F7E8883E7EDF0E067
:104DB00080818160808384E082BF81E08093DE0413
:104DC00088818E7F888302EE10E0F80110821092B5
:104DD000DA0081EEC82ED12CF601108288818F77FF
:104DE000888388818068888388818F7D888319BCC7
:104DF000109290021092910210928F0210928E02E5
:104E000090EEE92EF12CF70180818B7F80838881E1
:104E10008160888342E060E080E00E949426F60191
:104E200080818E7F8083F801808181608083808192
:104E300088608083F70180818E7F80838881806194
:104E40008883DF91CF911F910F91FF90EF90DF90BA
:104E5000CF9008951F920F920FB60F9211242F93A7
:104E60003F934F935F936F937F938F939F93AF93F2
:104E7000BF93EF93FF938091E10082FF09C080917F
:104E8000E20082FF05C08091E1008B7F8093E1000A
:104E90008091DA0080FF2AC08091D80080FF26C070
:104EA0008091DA008E7F8093DA008091D90080FFB4
:104EB00018C080E189BD82E189BD09B400FEFDCF43
:104EC00081E0809390028091DE0481110FC00E94E6
:104ED00023260E94C9268091E20084608093E2002C
:104EE00005C019BC109290021092DE048091E1007E
:104EF00080FF17C08091E20080FF13C08091E20024
:104F00008E7F8093E2008091E20080618093E200D6
:104F10008091D80080628093D80019BC85E080938E
:104F200090028091E10084FF45C08091E20084FFFF
:104F300041C080E189BD82E189BD09B400FEFDCF99
:104F40008091D8008F7D8093D8008091E1008F7E82
:104F50008093E1008091E2008F7E8093E200809157
:104F6000E20081608093E20080919102882311F039
:104F700084E007C08091E30087FD02C081E001C0AA
:104F800083E08093900210926B020E94A4250E94FD
:104F9000EF081092E5048091E404882349F08091A1
:104FA000DF0481608093DF0460E086950E94D90E63
:104FB0000E94C30E8091E10083FF27C08091E20030
:104FC00083FF23C08091E100877F8093E10082E02E
:104FD00080939002109291028091E1008E7F8093E5
:104FE000E1008091E2008E7F8093E2008091E200F8
:104FF00080618093E20042E060E080E00E949426BD
:105000008091F00088608093F000FF91EF91BF9154
:10501000AF919F918F917F916F915F914F913F9150
:105020002F910F900FBE0F901F901895209198020E
:10503000309199022617370748F06115710539F448
:105040002091E8002E772093E80001C0B901FC010F
:1050500020E06115710579F1809190028823F1F1CA
:105060008530F1F18091E80083FD3CC08091E8003B
:1050700082FD2EC08091E80080FFEBCF2091F300ED
:105080008091F20090E0922B6115710551F088300B
:10509000910538F421912093F10061507109019636
:1050A000F3CF21E0089709F020E08091E8008E77A7
:1050B0008093E800CECF2111CFCF0AC0809190021B
:1050C000882361F0853061F08091E80083FD0AC09B
:1050D0008091E80082FFF2CF80E0089582E0089599
:1050E00083E0089581E008958091DD04811107C077
:1050F00080919002843011F081E0089582E008955B
:105100008823B1F19CEF980F913A30F4682F81E237
:1051100092E00E94CE1C14C090E2980F983090F458
:10512000877021E030E0A90102C0440F551F8A9525
:10513000E2F7CA01809590916B02892380936B02FC
:105140000C94E41D9BE5980F933020F480E090E0F0
:105150000C94D90898E5980F973120F480E090E0FE
:105160000C94C308803F20F00E94011B0C948F1CFC
:105170000895882309F4CAC09CEF980F913A30F43F
:10518000682F81E292E00E94F61C13C090E2980F13
:10519000983088F4877021E030E0A90102C0440F04
:1051A000551F8A95E2F7CA0190916B02892B809373
:1051B0006B020C94E41D9BE5980F933070F4853AD4
:1051C00029F0863A31F083E890E005C081E890E06C
:1051D00002C082E890E00C94D90898E5980F9731C6
:1051E00008F08EC0883A09F445C0893A09F445C0F0
:1051F0008A3A09F445C08B3A09F445C08C3A09F45F
:1052000045C08B3B09F445C08C3B09F445C08D3A41
:1052100009F445C0803B09F445C08E3A09F445C005
:105220008F3A09F445C0813B09F445C0823B09F43B
:1052300045C0833B09F445C0843B09F445C0853B28
:1052400009F445C0863B09F445C0873B09F445C0D5
:10525000883B09F445C0893B09F445C08D3B09F4FE
:1052600045C08E3B09F445C08A3B09F445C080E047
:1052700090E044C082EE90E041C089EE90E03EC0F4
:105280008AEE90E03BC085EB90E038C086EB90E082
:1052900035C083EB90E032C084EB90E02FC087EB09
:1052A00090E02CC08CEC90E029C08DEC90E026C002
:1052B00083E891E023C08AE891E020C082E991E090
:1052C0001DC084E991E01AC081E292E017C083E238
:1052D00092E014C084E292E011C085E292E00EC038
:1052E00086E292E00BC087E292E008C08FE690E091
:1052F00005C080E790E002C08AE292E00C94C30807
:10530000803F20F00E94CB1B0C948F1C08958EE1EF
:105310004A9B02C08150E1F74A9BFECF08955A98FC
:1053200080E28A95F1F75A9A0895FC012AE02A95BD
:10533000F1F790E020E080E031E0261779F040E1DD
:105340004A95F1F7880F4A9B02C08160932700C0FD
:10535000000040E14A95F1F72F5FEFCF20E12A9559
:10536000F1F729B100C0000030E13A95F1F722FBD6
:10537000222720F992272081920F90830895EF929F
:10538000FF920F931F93CF93DF931F92CDB7DEB79A
:1053900019828C017C01E60EF11C0E151F0559F0D7
:1053A0000E94872968E0CE0101960E949529F801A4
:1053B00081938F01F2CF81E09981911180E00F906C
:1053C000DF91CF911F910F91FF90EF9008959093EF
:1053D000E8048093E7046093E604529A5A9A089589
:1053E0009093E8048093E7046093E60452985A9AF5
:1053F000EA9AE9E6F0E080818F7C8083089561502D
:1054000091E001C0990F6A95EAF720E031E0992315
:1054100061F0492F482319F05A9A232701C05A985E
:1054200040E24A95F1F79695F2CF222311F05A9A6D
:1054300001C05A9880E28A95F1F75A980895FF9230
:105440000F931F93CF93DF93EC018C01060F111D77
:10545000C017D10741F0F9900E948F2968E08F2D85
:105460000E94FF29F5CFDF91CF911F910F91FF90FF
:1054700008951F920F920FB60F9211240F931F934E
:105480002F933F934F935F936F937F938F939F934C
:10549000AF93BF93EF93FF93CF93DF931F92CDB75B
:1054A000DEB719820E94872967E0CE0101960E942B
:1054B0009529382F369536953695932F9695957074
:1054C000232F2570920F292F23709695969587701C
:1054D000920F891348C08981811145C08091E604EB
:1054E000831708F440C080E18A95F1F75A9A529ADE
:1054F000A2E0AA95F1F700C00091E7041091E8043A
:10550000B8E03B9F000D111D11245A98F8016581E8
:10551000662321F0868197810E941F2A0E948F298D
:10552000F0E1FA95F1F75A9852985A9A80E18A95E3
:10553000F1F7D80112966C911297662369F01396D1
:105540008D919C9114970E94BF29D801ED91FC91F7
:10555000811105C082E004C0D801ED91FC9188E082
:1055600080830E9487290F90DF91CF91FF91EF9167
:10557000BF91AF919F918F917F916F915F914F916B
:105580003F912F911F910F910F900FBE0F901F9081
:1055900018950F931F93CF93DF932091E60430E08B
:1055A000281739070CF471C09C0193E0220F331FB8
:1055B0009A95E1F7C091E704D091E804C20FD31F98
:1055C000F894529A5A9845E04A95F1F70000982FBE
:1055D000969595708570890F982F9370869586950E
:1055E000890F8901082B0E948F2984E08A95F1F7A1
:1055F00000C067E0802F0E94FF2940E14A95F1F743
:1056000052985A9A4A9902C000C0FCCF87E090E0B5
:105610004A9B0EC0019751F4529A5A9AE881F98137
:1056200081E08083789481E090E031C000C0F0CFC9
:105630006D81662381F08E819F810E94BF29811137
:105640000AC0529A5A9AE881F98182E0808378945C
:1056500082E090E01CC00E94872980E28A95F1F7E1
:105660005A98529A40E14A95F1F76A81662321F0EF
:105670008B819C810E941F2A0E948F29E881F981D9
:105680001082789480E090E002C084E090E0DF91A6
:10569000CF911F910F9108951092B9008CE08093E3
:1056A000B8000895EF92FF920F931F93CF93DF936B
:1056B000182FEB011092BC0084EA8093BC000E947A
:1056C000831C7C018091BC0087FD0EC0CF3F8FEF13
:1056D000D807C1F30E94831C8E199F098C179D0760
:1056E00088F38EEF9FEF2EC08091B900887F8830BD
:1056F00041F08091B900887F803119F08FEF9FEFE2
:1057000021C01093BB0084E88093BC000E94831CDE
:105710008C018091BC0087FD0CC0CF3F8FEFD80774
:10572000C1F30E94831C801B910B8C179D0788F38B
:10573000D8CF8091B900887F883111F08034F1F69C
:1057400080E090E0DF91CF911F910F91FF90EF905B
:1057500008950F931F93CF93DF93EB018093BB00CA
:1057600084E88093BC000E94831C8C018091BC0063
:1057700087FD0EC0CF3F8FEFD807C1F30E94831C77
:10578000801B910B8C179D0788F38EEF9FEF0CC049
:105790002091B900287F81E090E0283211F480E068
:1057A00090E0919581959109DF91CF911F910F9193
:1057B0000895CF92DF92EF92FF920F931F93CF93B2
:1057C000DF936B018A017901B9010E94522BE60136
:1057D0000C0D1D1DC017D10761F424E92093BC00F6
:1057E000DF91CF911F910F91FF90EF90DF90CF90BD
:1057F000089597FDF2CFB70189910E94A92BEACFB6
:10580000CF92DF92EF92FF920F931F93CF93DF938C
:10581000C62F6A017901B8010E94522B97FD11C071
:10582000B8018C2F0E94A92BE601EC0CFD1CCE15B3
:10583000DF0539F097FD05C0B80189910E94A92BB9
:10584000F6CF24E92093BC00DF91CF911F910F91F7
:10585000FF90EF90DF90CF90089584E98093BC0093
:105860000895FB01DC0102C005900D9241505040AB
:10587000D8F70895F999FECF92BD81BDF89A99277E
:1058800080B50895A6E1B0E044E050E00C94742C9B
:10589000A8E1B0E042E050E00C94742C262FF99976
:1058A000FECF92BD81BDF89A019700B4021639F07F
:1058B0001FBA20BD0FB6F894FA9AF99A0FBE089550
:1058C0000396272F0E944F2C0E944E2C252F0E94BA
:1058D0004F2C242F0C944F2C0196272F0E944F2CD5
:1058E0000C944E2CDC01CB01FC01F999FECF06C0D3
:1058F000F2BDE1BDF89A319600B40D92415050408E
:10590000B8F70895991B79E004C0991F961708F01D
:10591000961B881F7A95C9F780950895AA1BBB1B13
:1059200051E107C0AA1FBB1FA617B70710F0A61B9F
:10593000B70B881F991F5A95A9F780959095BC01C0
:10594000CD01089597FB072E16F4009407D077FD3C
:1059500009D00E948E2C07FC05D03EF490958195CD
:105960009F4F0895709561957F4F0895EE0FFF1F2B
:105970000590F491E02D0994FC014150504030F025
:1059800001900616D1F73197CF01089588279927FE
:105990000895FB01DC0104C08D910190801921F470
:1059A00041505040C8F7881B990B0895F894FFCFD9
:1059B00005FFFF0101C00100000001BF01C001049B
:1059C000BB0101BF01BA0100000004B601002100C3
:1059D0007F2200038C1ABA1A8F1A39156F15019499
:1059E0006697C600000000000102020202060606D9
:1059F000090909090909F4F5F6F7313332000810ED
:065A000018181008000058
:00000001FF
